:05000000020033814401
:02000B0081452D
:02001300814624
:02001B0081471B
:02002300814812
:02002B00814909
:10003300759840758780758921758DFF758BFF7560
:100043008840D2997581607530007531007535FF30
:10005300D210D211D212D213D214D215D216D21771
:10006300D218D219D21AD21BD21CD21DD21ED21F21
:10007300D220D221D222D223D234D235D236D23791
:10008300C2B0D2A27407B535037535FF0535E53522
:10009300A2E092A4A2E192A5A2E292A6D2A7D29054
:1000A300209014301021C210B211201105120464E3
:1000B300801512047F801020100DD210201105121C
:1000C300047B8003120496C2A7D2912091143012AC
:1000D30021C212B21320130512049A80151204B51B
:1000E300801020120DD2122013051204B1800312C6
:1000F30004CCD292209214301421C214B2152015CC
:10010300051204D080151204EB801020140DD214B4
:100113002015051204E78003120502D293209314DD
:10012300301621C216B217201705120506801512C4
:100133000521801020160DD21620170512051D80EB
:1001430003120538D294209414301821C218B2191E
:1001530020190512053C8015120557801020180D33
:10016300D218201905120553800312056ED295206B
:100173009514301A21C21AB21B201B051205728076
:100183001512058D8010201A0DD21A201B05120599
:100193008980031205A4D296209614301C21C21C18
:1001A300B21D201D051205A880151205C38010205D
:1001B3001C0DD21C201D051205BF80031205DAD2C7
:1001C30097209714301E21C21EB21F201F0512054F
:1001D300DE80151205F98010201E0DD21E201F058A
:1001E3001205F58003120610D2A020A0143020219E
:1001F300C220B221202105120614801512064C805C
:100203001020200DD2202021051206308003120673
:1002130068D2A120A114302221C222B223202305B7
:1002230012068480151206A4801020220DD22220EB
:1002330023051206A080031206C0D2B220B21430E6
:100243003421C234B2352035051206C48015120696
:10025300E4801020340DD2342035051206E08003EB
:10026300120700D2B320B314303621C236B237207E
:100273003705120704801512071F801020360DD290
:100283003620370512071B8003120736D2B420B479
:100293001C75320712073A12044AD5320675320129
:1002A30012073A120451D2B420B40280EDD2B52021
:1002B300B51C75320712075012044AD5320675323F
:1002C30001120750120451D2B520B50280EDD2B607
:1002D30020B61C75320712076612044AD53206751A
:1002E3003201120766120451D2B620B60280EDD253
:1002F300B720B71C75320712077F12044AD532069E
:1003030075320112077F120451D2B720B70280ED74
:10031300E4B53502613F04B53502615F04B53502CA
:10032300617F04B53502619F04B5350261BF04B531
:10033300350261DF04B5350261FF811FE580F536C3
:10034300A837A936120458400624FE500D80051222
:10035300045D5006853637120798813FE580F538EE
:10036300A839A938120458400624FE500D800512FE
:10037300045D50068538391207B4813FE580F53AAC
:10038300A83BA93A120458400624FE500D800512DA
:10039300045D5006853A3B1207D0813FE580F53C6A
:1003A300A83DA93C120458400624FE500D800512B6
:1003B300045D5006853C3D1207EC813FE580F53E28
:1003C300A83FA93E120458400624FE500D80051292
:1003D300045D5006853E3F120808813FE580F540E5
:1003E300A841A940120458400624FE500D8005126E
:1003F300045D5006854041120824813FE580F542A3
:10040300A843A942120458400624FE500D80051249
:10041300045D5006854243120840813FE580F54460
:10042300A845A944120458400624FE500D80051225
:10043300045D5006854445120854813F0183020040
:10044300333232323232327E20DFFEDEFC227E60F5
:10045300DFFEDEFC22C2D7E89922C2D7E99824FE48
:10046300223099FDC2997599C03099FDC299759949
:100473000075300012044A2212044A223099FDC248
:10048300997599C03099FDC299759900753000121C
:10049300044A2212044A223099FDC2997599C03048
:1004A30099FDC29975990175300112044A2212040B
:1004B3004A223099FDC2997599C03099FDC2997548
:1004C300990175300112044A2212044A223099FD1F
:1004D300C2997599C03099FDC29975990275300218
:1004E30012044A2212044A223099FDC2997599C016
:1004F3003099FDC29975990275300212044A22128D
:10050300044A223099FDC2997599C03099FDC29968
:1005130075990375300312044A2212044A22309952
:10052300FDC2997599C03099FDC2997599037530CB
:100533000312044A2212044A223099FDC299759982
:10054300C03099FDC29975990475300412044A228A
:1005530012044A223099FDC2997599C03099FDC29F
:100563009975990475300412044A2212044A223000
:1005730099FDC2997599C03099FDC2997599057510
:10058300300512044A2212044A223099FDC2997599
:1005930099C03099FDC29975990575300512044AC1
:1005A3002212044A223099FDC2997599C03099FDEF
:1005B300C29975990675300612044A2212044A221A
:1005C3003099FDC2997599C03099FDC29975990604
:1005D30075300612044A2212044A223099FDC29948
:1005E3007599C03099FDC299759907753007120442
:1005F3004A2212044A223099FDC2997599C0309952
:10060300FDC29975990775300712044A2212044AEC
:10061300223099FDC2997599B03099FDC2997599A7
:10062300403099FDC29975997F12044A223099FD91
:10063300C2997599B03099FDC2997599403099FD69
:10064300C29975990012044A223099FDC29975998D
:10065300B03099FDC2997599403099FDC299759949
:100663007F12044A223099FDC2997599B03099FDE1
:10067300C2997599403099FDC29975990012044A3F
:10068300223099FDC2997599B03099FDC299759937
:10069300413099FDC29975997F12044A2212044A86
:1006A300223099FDC2997599B03099FDC299759917
:1006B300413099FDC29975990012044A2212044AE5
:1006C30022E53004B40801E4F5303099FDC2997590
:1006D30099C03099FDC299F59912044A2212044A2D
:1006E30022E53004B40801E4F5303099FDC2997570
:1006F30099C03099FDC299F59912044A2212044A0D
:10070300223099FDC2997599C03099FDC2997599A6
:100713000175300112044A2212044A223099FDC2A3
:10072300997599C03099FDC2997599007530001279
:10073300044A2212044A223099FDC2997599C030A5
:1007430099FDC2990531E531547FF599223099FD20
:10075300C2997599C03099FDC2991531E531547F1D
:10076300F599223099FDC2997599B03099FDC299D6
:100773007599603099FDC299759900223099FDC22F
:10078300997599B03099FDC2997599613099FDC2F7
:1007930099759900223099FDC2997599B03099FDE8
:1007A300C2997599053099FDC299E536C313F59938
:1007B300223099FDC2997599B03099FDC299759906
:1007C300023099FDC299E538C313F599223099FD9A
:1007D300C2997599B03099FDC2997599013099FD07
:1007E300C299E53AC313F599223099FDC2997599D7
:1007F300B03099FDC29975990B3099FDC299E53CCA
:10080300C313F599223099FDC2997599B03099FDBA
:10081300C29975990A3099FDC299E53EC313F599BA
:10082300223099FDC2997599B03099FDC299759995
:10083300073099FDC299E540C313F599223099FD1C
:10084300C2997599D03099FDC299E542C313F599C0
:10085300223099FDC2997599E03099FDC299759935
:10086300003099FDC299E544C313F59922204D75D3
:100873007A796B616E7420352076312E30622032A6
:100883003030372D30322D323720286329416461CF
:100893006D20536D69616C656B206A616E6B6F6D62
:1008A300757A796B616E744077702E706C207777F0
:1008B300772E736D69616C656B2E7072762E706C1A
:1008C3002057737A656C6B6965207072617761205C
:1008D3007A617374727A657A6F6E652E204A616BE2
:1008E30069656B6F6C7769656B207A6173746F737D
:1008F3006F77616E6961206B6F6D657263796A6E84
:1009030065206B6F6475206E6965646F7A776F6CB1
:100913006F6E652E20416C6C20526967687473207A
:1009230052657365727665642E204672656520662E
:100933006F72206E6F6E20636F6D6D657263696198
:080943006C206F6E6C792E2010
:00000001FF
